:020000040000FA
:04000000ADEF08F068
:08000800056ED8CF06F0E0CF31
:1000100007F00001E9CF0DF0EACF08F0E1CF09F0D9
:10002000E2CF0AF0D9CF0BF0DACF0CF0F3CF14F017
:10003000F4CF15F0FACF16F000C00FF001C010F0A9
:1000400002C011F003C012F004C013F0F2AA2CEFAA
:1000500000F0F2B470EF07F0A0AA32EF00F0A1BAFE
:100060003BEF07F00FC000F010C001F011C002F02C
:1000700012C003F013C004F00E8E0DC0E9FF08C0DB
:10008000EAFF09C0E1FF0AC0E2FF0BC0D9FF0CC0C4
:10009000DAFF14C0F3FF15C0F4FF16C0FAFF0550D5
:1000A00007C0E0FF06C0D8FF1000F76ABA0FF66E6F
:1000B000000EF7220900F5501200040301000000B1
:1000C00000000000000000000000F76ADA0FF66E82
:1000D000000EF7220900F550120004000100000094
:1000E00000000000000000000000F76AFA0FF66E42
:1000F000000EF7220900F5501200400008004000F1
:1001000000000000000000000000000000000000EF
:1001100000000000000000000000F76A2A0FF66EE1
:10012000010EF7220900F5501200400000004000C7
:1001300000000000000000000000000000000000BF
:1001400000000000000000000000F76A5A0FF66E81
:10015000010EF7220900F5501200090243000201C6
:1001600000C0320904000001020201000524001051
:1001700001042402020524060001052401000107F0
:100180000581030800FA09040100020A00000007C3
:100190000502024000FA070582024000FA00F76AF1
:1001A000AE0FF66E010EF7220900F55012000200A4
:1001B000F76AC00FF66E010EF7220900F550120023
:1001C000120110010200004061043300000101022D
:1001D0000001F76AE20FF66E010EF7220900F550F2
:1001E00012000403090408034300430053001E03E4
:1001F00043004300530020005200530032003300FC
:1002000032002000440065006D006F00F2CF0EF058
:10021000F29EF76A260FF66E020EF7220900F550DD
:100220000EBEF28E12000D0A0D0A4C6F616420435F
:10023000656C6C20414443202863293230303820DB
:100240002E737465656D616E2E62650D0A00F2CFC6
:100250000EF0F29EF76A680FF66E020EF7220900A2
:10026000F5500EBEF28E12002057616974696E67F8
:1002700020666F722069676E6974696F6E2C2073D7
:100280007769746368206F6E207465787420636189
:100290007074757265206E6F77200D0A0D0A00006C
:1002A000F2CF0EF0F29EF76ABA0FF66E020EF72248
:1002B0000900F5500EBEF28E120053616D706C6530
:1002C0002073706565643A20256C6420487A202D7F
:1002D00020426173652076616C75653A20256C64F7
:1002E0002041444320626974730D0A006D92699441
:1002F000689446EF07F06A6A68924FEF07F02C6A3D
:100300002B6A250E2A6E800E296E2D6A2E6A080E23
:100310002F6E7F6B7A93316A306A7B6B7C917A8126
:10032000000CA66BA65101080AE3036AA651270F29
:10033000E96E000E0320EA6EEF6AA62BF3D7DFDF2B
:100340001A6A010E1B6E196A000C010EAF6FAF51D5
:100350000F080EE3700EAF25016E0F0E036ED8B0BE
:10036000032A01C0E9FF03C0EAFFEF6AAF2BEFD712
:100370001E6A1D6A000C400E0401016F050E036F1A
:10038000026B880E006F046B050E076F400E066F40
:100390000001000C6A6A686A9F0E6B6E390E696E06
:1003A0006E6ABFDFD2DF160E706E68A602D0689646
:1003B000FCD76D98E0DF030E1F6E55EF07F06984E0
:1003C00068986D825BEF07F0689C61EF07F070A0A2
:1003D00002D0D1DF7090689A67EF07F0AAC020F0D2
:1003E000000CFF0E206E000CA86B265235E0A851C1
:1003F0003F0832E31C5005E0020A0DE0010A15E057
:100400001ED0036A2550F2CFAAF0F29E9EDEAABF4C
:10041000F28EA96F14D0036A2550F2CFAAF0F29E93
:10042000D8DEAABFF28EA96F0AD0036A2550F2CF98
:10043000AAF0F29EBDDEAABFF28EA96F00D0252AD7
:100440002606A851A82B036A400FE96E050E03206B
:10045000EA6EA9C0EFFFC9D7265204E1A8514008AF
:1004600001E0196AA8C0AAF0B9DF000C256A1C6A6D
:1004700005010351010A000105E0030A08E0010A31
:1004800009E01FD0120E266E030E1C6E1CD0430E08
:10049000266E19D0020E1C6E036A05010251210F4F
:1004A000E96E000E0320EA6EEFCF25F0036A2550B7
:1004B000F2CFA7F0F29E00018CDEA7BFF28E266E6F
:1004C00002D08FDF0CD00501075305E12650065DF1
:1004D00002E206C526F0010E196E000185DF89EFE4
:1004E00003F0A75304E1040E1F6E2FDFC1D0050EE9
:1004F0001F6EAA6F800EA96F010EA86FA8510F087A
:10050000D8A0B6D0AB6B036AA851F2CFAFF0F29E81
:10051000DCDDAFBFF28E000A51E0040EAB6FD89065
:10052000A835036AF2CFAFF0F29EF7DD0900F5CFF0
:1005300003F0AFBFF28EAC6F03C0ADF0A851080D51
:10054000F350010F016E040E036ED8B0032A01C0F0
:10055000E9FF03C0EAFFACC0EFFFA851080DF3505C
:10056000020F016E040E036ED8B0032A01C0E9FF2A
:1005700003C0EAFFAAC0ECFFED52A9C0EFFFD8907C
:10058000A835036AF2CFAFF0F29EC7DD0900F5CFC0
:1005900003F0AFBFF28EA9270350AA23880EAE6FD7
:1005A000ADB1AE81ADB3AE83A851080DF3CF01F06C
:1005B000040E01C0E9FFEA6EAEC0EFFF036AA85166
:1005C000F2CFAFF0F29E71DDAFBFF28E000A31E0E4
:1005D000AB83A851080DF350060F016E040E036E95
:1005E000D8B0032A01C0E9FF03C0EAFFAAC0ECFFAC
:1005F000ED52A9C0EFFFD890A835036AF2CFAFF053
:10060000F29E73DD0900F5CF03F0AFBFF28EA9278C
:100610000350AA23A851080DF350040F016E040ED5
:10062000036ED8B0032A01C0E9FF03C0EAFF400E01
:10063000EF6EAB51060802E10E0EAB6F036AA851D4
:10064000F2CFAFF0F29E31DDAFBFF28E020801E0D3
:10065000AB89700EA825016E0F0E036ED8B0032A69
:1006600001C0E9FF03C0EAFFABC0EFFFA82B46D7EC
:1006700083EF03F00501015100010DE0010A14E0D0
:10068000020A1EE0060A27E0030A2CE00E0A2BE00D
:10069000010A2FE03CD01BC040F50501416B020E62
:1006A0000001AA6F9BDE35D00501022D06D0010E98
:1006B0001B160001AA6B92DE02D0000192DE29D047
:1006C0000501022D05D01B820001AA6B87DE02D036
:1006D000000187DE1ED0020E196E02C524F0AA6B3F
:1006E0007DDE17D0C3D61AC040F5010EAA6F76DEA4
:1006F00010D005010251010808E302C51AF002C535
:10070000A7F00001EED6AA6B69DE000102D069DE17
:1007100000D001EF05F01AC0A7F00501015100015A
:1007200005E00A0A0BE0010A2BE03CD00501406B12
:10073000416B020E0001AA6F51DE36D0A7531EE0B6
:10074000010EA75D036AF2CFA9F0F29E28DDA9BFD2
:10075000F28E016E0501045DD8A002D000010ED01A
:10076000036A0451270FE96E000E0320EA6EEFCFF3
:1007700040F5010E0001AA6F31DE01D032DE14D047
:10078000A7530EE0036A05010451270FE96E000E1E
:100790000320EA6E02C5EFFF0001AA6B1FDE01D045
:1007A00020DE02D01EDE00D001EF05F0A891A7BF29
:1007B000A881A79FA8A110D0036AA751F2CFA9F0E2
:1007C000F29E73DCA9BFF28E000A02E1000E01D096
:1007D000010E016E10D00FD0036AA751F2CFA9F01D
:1007E000F29E73DCA9BFF28E000A02E1000E01D076
:1007F000010E016E00D06DEF04F0A891A7BFA88193
:10080000A79FA8A110D0A751080DF350040F016EA7
:10081000040E036ED8B0032A01C0E9FF03C0EAFF4B
:10082000880EEF6E09D0A751080DF3CF01F0040E2A
:1008300001C0E9FFEA6EEF6A7CEF04F0A891A7BF60
:10084000A881A79FA8A110D0A751080DF350040FAD
:10085000016E040E036ED8B0032A01C0E9FF03C085
:10086000EAFF840EEF6E0AD0A751080DF3CF01F016
:10087000040E01C0E9FFEA6E840EEF6E82EF04F011
:10088000A891A7BFA881A79FA8A110D0A751080D24
:10089000F350040F016E040E036ED8B0032A01C09A
:1008A000E9FF03C0EAFFEFCFA9F00AD0A751080D76
:1008B000F3CF01F0040E01C0E9FFEA6EEFCFA9F01B
:1008C000A9AF02D0A9B502D0000E01D0010E016E71
:1008D0008CEF04F004C5A7F069D7015229E00501A7
:1008E0000151010A000105E0020A09E0030A0DE0D6
:1008F0001DD004C5A7F081D7AA6B70DD19D004C53F
:10090000A7F09CD7AA6B6ADD13D00501406B416B41
:1009100004C5A7F00001B4D7015204E0010E05019F
:10092000406F0001020EAA6F59DD02D05ADD00D0DF
:1009300001EF05F0FE0E206E000C0501042D01D024
:1009400002D0045348E1015100010BE0010A0DE01F
:10095000210A1CE0010A1FE0030A2EE0010A31E02F
:1009600037D0010E806FE6DF35D0050EEA6E400EFF
:10097000E96EE26A320EE16E080E016EE6CFEEFF1E
:10098000012EFCD706C5AAF029DD24D0020E806F07
:100990007A83D0DF1FD0050EEA6E400EE96EE26A60
:1009A000290EE16E070E016EE6CFEEFF012EFCD799
:1009B000070EAA6F13DD0ED002C57FF0AA6B0EDD05
:1009C00009D002C531F003C530F0AA6B07DD02D0B3
:1009D00008DD00D00501000101EF05F0196A0501ED
:1009E00000517F0B000107E0010A06E0030A05E061
:1009F000230A04E004D03ED68ED66CD79ED7F1DC15
:100A000000D0E6EF06F0A751080DF3CF01F0040E79
:100A100001C0E9FFEA6EEFCFA9F0A851020806E194
:100A2000A9AD02D0A86B02D0010EA86FA85103088F
:100A300012E1840EA96FA751080DF350040F016E47
:100A4000040E036ED8B0032A01C0E9FF03C0EAFF19
:100A5000840EEF6E09D0A82D03D0C80EA96F04D064
:100A6000A85302E1880EA96F036A010E026EA75116
:100A7000006E05E0D89002360336002EFBD70250F8
:100A8000FF0A006EFF0E031A00501D1603501E16BB
:100A9000D890A735036AF2CFACF0F29E8DEC00F04F
:100AA0000900F5CF03F0ACBFF28EAA6F03C0ABF024
:100AB000A751080DF350010F016E040E036ED8B05C
:100AC000032A01C0E9FF03C0EAFFAAC0EFFFABB1F0
:100AD000A981ABB3A983A751080DF3CF01F0040E90
:100AE00001C0E9FFEA6EA9C0EFFF000CB351080D89
:100AF000F350040F016E040E036ED8B0032A01C038
:100B0000E9FF03C0EAFFEFCFB7F0B7BF5BD0B35147
:100B1000080DF350050F016E040E036ED8B0032AC2
:100B200001C0E9FF03C0EAFFB4C0EFFFB6510208FD
:100B300016E1B351080DF350040F016E040E036E5D
:100B4000D8B0032A01C0E9FF03C0EAFFEFCFB7F036
:100B5000B7AD02D0B66B02D0010EB66F13D0B6514E
:100B6000040810E1B351080DF3CF01F0040E01C0E9
:100B7000E9FFEA6EEFCFB7F0B7AD03D0010EB66F65
:100B800001D0B66BB62D03D0C80EB76F04D0B653E4
:100B900002E1880EB76FB5B1B781B5B3B783B35172
:100BA000080DF350040F016E040E036ED8B0032A33
:100BB00001C0E9FF03C0EAFFB7C0EFFF010E016EFD
:100BC00003D000D0000E016E000C8051010A03E03A
:100BD000030A12E022D0EA6A320EE96E050EE26ED6
:100BE000E16A080E016EE6CFEEFF012EFCD7AA6B7C
:100BF000EEEC01F0806B15D0EA6A290EE96E050E65
:100C0000E26EE16A070E016EE6CFEEFF012EFCD721
:100C1000806BAA6BEEEC01F004D0806BBBEC01F0B2
:100C200000D033EF06F0A851080DF350010F016E0C
:100C3000040E036ED8B0032A01C0E9FF03C0EAFF27
:100C4000036AEFCF01F003C002F02CEF06F07C81C5
:100C50007E6B020EA86FE7D701C07DF038EF06F07B
:100C6000A75302E1B2D714D0A751020802E1EFD78F
:100C70000FD0036A010E026EA751006E05E0D890F6
:100C800002360336002EFBD702501D1203501E12EF
:100C9000000CA8C06EFFA85303E0040E1F6E02D024
:100CA000020E1F6E59EF06F01A6A196A24C0A8F0E6
:100CB000F0D7D0EF06F0A851080DF350040F016EE5
:100CC000040E036ED8B0032A01C0E9FF03C0EAFF97
:100CD000EFCFB0F0B0BF3FD0A851080DF350060FD2
:100CE000016E040E036ED8B0032A01C0E9FF03C0F1
:100CF000EAFFECCF03F0ED52EFCFB1F003C0B2F05A
:100D0000AF6BAE6BAF51AC5D1AE303E1AB51AE5DBF
:100D100016E2A9C0E9FFAAC0EAFFEFCFB5F0B2C062
:100D2000EAFFB1C0E9FFB5C0EFFFB12BD8B4B22BD9
:100D3000A92BD8B4AA2BAE2BD8B4AF2BE3D7A8C01D
:100D4000B3F0ACC0B5F0ABC0B4F0ADC0B6F0CEDE21
:100D5000015003D000D0000E016E000C7B530DE05B
:100D60007A91020EA86FAA6B3A0EA96FAC6B7BC08A
:100D7000ABF0020EAD6F9FDF7B6B000C7B5302E08C
:100D8000EDDF01D07A81D5EF06F0A7530AE1192CE7
:100D900003D0F4EC01F004D01950020801E184D72B
:100DA00004D0A751020801E1E9D7000C6C30A66F0E
:100DB000A633A6331F0EA6176C523BE10401005167
:100DC0003C0B34081BE1046B000108D6203C05D025
:100DD000A76B030EA86F17DE0ED0A76B020EA86FCD
:100DE00012DE2050FE0807E0B36BB56B20C0B4F0F4
:100DF000040EB66F7BDE6D9819D0040100513C0BD8
:100E0000040815E10001A76B2BDFA76B020EA86F8A
:100E1000FADD2050FE080AE0203C01D007D0B36B79
:100E2000B56B20C0B4F0010EB66F60DE040120D0B7
:100E300000016C50040812E1FF0E206EA76BA5DFC5
:100E4000203C01D008D0B36BB56B20C0B4F0020ECB
:100E5000B66F4CDE02D0BBEC01F009D06CB404D00C
:100E6000A6C0A7F0FDDE03D0A6C0A7F08EDF040168
:100E700000016CEF07F01F5201E12FD068522DE006
:100E800068A404D069A402D076EF01F06DA201D06D
:100E900024D068A204D069A202D07BEF01F068A040
:100EA00004D069A002D0CAEF01F068A804D069A8F4
:100EB00002D0DFEF01F068AC04D069AC02D0E4EFFF
:100EC00001F068AA04D069AA02D0E7EF01F068A691
:100ED00004D069A602D06AD76896A19A32EF00F0D2
:100EE000C282C2B2FED7C3CF81F0C4CF82F0830EDC
:100EF000D6267A85F29432EF00F06D6A696A080EA0
:100F00006F6E94503009946E1F6A186AF2BE188E84
:100F1000F29E91EC01F018BEF28E1E6A1D6AB4EFCB
:100F200007F0186AF2BE188EF29E91EC01F018BE1E
:100F3000F28E6D6A140E6F6E696A6D86010E1F6EF9
:100F4000A5EF07F06DB601D0ECD71F2C0BD06DBA12
:100F500009D0686A696AA08AC00EF212110E696E21
:100F6000020E1F6E000CC9D7EDDF1F500208FCE116
:100F7000CEEF07F0C30ED56EC150C00B0E09C16E87
:100F8000C080C082C084C08EC280000E016EC2507C
:100F9000C30B0110C26E7FEC01F0E5D7C8EF08F07B
:100FA000EA6A860EE96EEF500EE00F0E016E006ADF
:100FB000002EFED7012EFBD78F0E006E002EFED71F
:100FC0000000EF2EF2D7000C9391F2BE9381F29EB7
:100FD0007B513F0802E23F0E7B6F7B517B2B036A04
:100FE0003A0FE96E000E0320EA6E92C0EFFFF29E08
:100FF00093B1F28E7AA107D0186AF2BE188EF29ED3
:10100000ADDE18BEF28E15EF08F07B513F080AE204
:101010007AA107D0186AF2BE188EF29E9FDE18BE23
:10102000F28EF3D791C092F0CFD7000C016A026A1A
:10103000006A036A895102E1885118E0100E8A6F34
:10104000D89086378737003603368951035C02E132
:101050008851005C07E38851005ED8A003068951DF
:10106000035ED880013602368A2FEAD73AEF09F0BC
:10107000EACF90F0E9CF8FF089AF08D08F8F8FA99A
:101080008F2B881F891F882BD8B4892B8939F009A9
:101090008B6F8B27E20F8C6F320F8E6F89510F0B86
:1010A0008C278C278E27E90F8D6F8D278D27883908
:1010B0000F0B8D278E278D378E378E1F8E378851D9
:1010C0000F0B8E278B37070E8A6F0A0E8D078E2720
:1010D000FDE38C078D27FDE38B078C27FDE38A0753
:1010E0008B27FDE3EA6A8A0EE96E070E8F158F9D46
:1010F000E9068F1507E18FB9E92A8FB903D0200ED1
:10110000006E1CD0E9268E0EE95CD8B48F8DEF50AE
:10111000006E08E18FBD06D08FB91BD08FB702D00B
:10112000200E0BD08FAF06D02D0E006EED508F9D90
:101130008F9F04D08F878F99300E0026EACF89F0D9
:10114000E9CF88F000C091F060DF89C0EAFF88C075
:10115000E9FFEE508FADD7D7000CF86AD09E0D8E08
:10116000EA6AE96AC150C00B0F09C16E070EB46E7E
:101170001F6A216A040E226E0C0E236E266A7B6B98
:10118000806B7A95816B826B836B846B7A97F2D6D6
:10119000640E866F05DF7AB306D0929A897A320E92
:1011A000866FFEDEF8D7929A899A866B865106EC96
:1011B00001F0862B006E916F28DF1A0E865DF6E136
:1011C000030E876F770E916F20DF872FFBD71A0EE4
:1011D000886F885106EC01F0882B006E916F15DF47
:1011E000270E885DF6E13E0E866F2D0E916F0DDFA6
:1011F000862FFBD70D0E916F08DF0A0E916F05DF6A
:10120000050E866F210E916F00DF862FFBD7876B4F
:10121000875127EC01F0872B006E916FF6DE320EBE
:10122000875DF6E1050E886F210E916FEEDE882F47
:10123000FBD7320E896F895127EC01F0892B006EA4
:10124000916FE3DE360E895DF6E1856B85516308AB
:1012500009E3C282C2B2FED7C3508327C45084239D
:10126000852BF4D784C087F083C086F0896B640E29
:10127000886FDCD602C084F001C083F0F28AC00E11
:10128000F21260DE1A5253E07AA551D0030E832584
:10129000016E000E8421036E0350825D38E303E18A
:1012A0008151015C34E27AB732D07A87866B8651FD
:1012B00050EC01F0862B006E916FA7DE0E0E865D5E
:1012C000F6E1100EE96E170E896F700E886FD0DE92
:1012D000110E876F875150EC01F0872B006E916FD4
:1012E00094DE230E875DF6E1100EE96E84C089F06E
:1012F00083C088F0BDDE260E886F885150EC01F067
:10130000882B006E916F81DE310E885DF6E17AA741
:101310000DD0100EE96E82C089F081C088F0A8DE81
:101320000D0E916F72DE0A0E916F6FDE7A95A9D75E
:021330000300B8
:020000040030CA
:0E000000240E3E1E008381000FC00FE00F4053
:00000001FF
